:020000040000FA
:100000008A150A1200280000F20003088301A000EC
:100010000A08A1000408A2008A150A120B191C2163
:100020000B1800008B180000831203138A110A12A8
:100030008C1960200C1B00008C1A00000C1A0000A8
:100040000C1900008C1800000C1800000D1800009E
:1000500083012208840021088A0020088300F20E10
:04006000720E090013
:1000C000831603171008110583128A110A120319E7
:1000D0008528AB008A110A122B19CF208A110A1227
:1000E0002B1889208A110A12AB19DB208A110A12F7
:1000F000AB1ABB208A110A12AB18C2208A110A124D
:100100002B1AAF208A110A126028831203138C1154
:100110000800AC01C4018316901190119011901148
:100120000830A100B830A2008830A000C030A6007E
:100130000830A40096019001831203138C118316DA
:100140000317063098003B309100FF3093000130D8
:10015000970083120130AD000313031708008316C4
:1001600011121012101111159514831203138C1112
:1001700003174414080083169012831203138C1182
:1001800003170800831690101208130592018312BA
:1001900003138C110317B000831203170800831692
:1001A00011111011101211169510831203138C11D6
:1001B0000317C40108008317831603171408A03E11
:1001C000840083120008A000840A0008A100840AA9
:1001D0000008A2008316031714089011831203135A
:1001E0008C110317C50020083C39B100243A8A114C
:1001F0000A12031928293108043A8A110A1203192C
:1002000008293108343A8A110A1203198A29080088
:1002100045088A110A12031D1D292E08213A8A1148
:100220000A12031D132983160830A1008830A0008C
:100230008A110A12831282290800083A8A110A12C6
:10024000031D232908004508103A03190800080077
:10025000450818398A110A12031D7B292E08063A0F
:100260008A110A12031D38298A110A127E247A295A
:100270002E08663A8A110A12031D44298A110A12AD
:100280007E248A110A127A292E08053A8A110A1246
:10029000031D50298A110A127B238A110A127A2916
:1002A0002E08033A8A110A12031D59298A110A12CB
:1002B0007A292E08013A8A110A12031D7729270884
:1002C000013A8A110A12031D6B298316191483122D
:1002D0008A110A127A292708023A8A110A12031D82
:1002E0007A2983161A1483128A110A127A298A111A
:1002F0000A126A2D0800083A8A110A12031D812980
:100300000800080083160317A501C830A400831253
:10031000AE0108008317220884000008A300840AA5
:100320000008A400840A0008A500840A0008A600AA
:10033000840A0008A700840A0008A800840A0008AC
:10034000A900840A0008AA0083160830A100A400AE
:1003500083122308213A88300319C8308316A0007D
:1003600015128312AE0123088A110A120319E82913
:100370002308013A8A110A120319032A2308023AB0
:100380008A110A120319182A2308803A8A110A12BC
:100390000319242A2308813A8A110A120319362ADA
:1003A0002308823A8A110A120319482A230860395D
:1003B000203A8A110A120319AD2C23086039403AF9
:1003C0008A110A12031D0C2B8A110A12AC2C080088
:1003D0002408013A8A110A120319872B2408053AC6
:1003E0008A110A1203196F2B2408093A8A110A127A
:1003F00003191C2C2408033A8A110A120319CB2B67
:100400008A110A120C2B2408013A8A110A120319C4
:10041000C82B24080B3A8A110A1203196B2C2408E2
:10042000033A8A110A1203190C2C8A110A120C2B96
:100430002408013A8A110A120319922B2408033A5C
:100440008A110A120319D62B2408083A8A110A12B3
:1004500003190F2C2408063A8A110A120319522A8A
:100460002408003A8A110A120319112B24080A3AA7
:100470008A110A1203194D2C2408003A8A110A1213
:100480000319202B2408063A8A110A120319522A4A
:100490002408003A8A110A1203194B2B8A110A12F6
:1004A0000C2B08002608223A8A110A120319012D82
:1004B0002608213A8A110A1203194F2D02308A00A8
:1004C000031026080339673E03188A0A82000C2BA2
:1004D0006B2A852AB52A0630AE000830B500933065
:1004E000B2000530B3008A110A128D25B400AA08A3
:1004F0008A110A12031D802A29022908031CB4004C
:10050000B40A8A110A127E2408000630AE000310D5
:10051000250D8A110A127925B2000310250D013E1E
:100520007925B3000230B2070318B30A8A110A1200
:100530008D25B4000230B202031CB303AA088A114D
:100540000A120319A62A8A110A12AE2A34082902AD
:100550008A110A120318AE2A2908B4000830B5001F
:10056000B40A8A110A127E2408006630AE002708F9
:100570008A110A12031DC62A2808031DC62A3F3005
:10058000B2000630B3008A110A12FD2A0630B30009
:100590004130B200BB018A110A120326B20A2702B7
:1005A0008A110A12031DDC2A8A110A120326280264
:1005B0008A110A120319E82AB20ABB0A453032022C
:1005C0008A110A12031CCB2AAE018A110A120C2BC3
:1005D000063025028A110A12031CF22AAE018A1182
:1005E0000A120C2B250DB3003B088A110A120926AA
:1005F000B200B30A3B080926B3008A110A12032687
:10060000B40029022908031CB4000830B500B40A5C
:100610008A110A127E240800831603171814831205
:100620000800831626088400831283172D08800093
:10063000840A800183160230A500C830A400080097
:1006400083161708023A8A110A12031D2D2B8312F2
:1006500027088A110A12031D2D2B83161708033A47
:100660008A110A12031D0C2B83122708003C8A11E1
:100670000A12031C0C2B2708383E8400831700083D
:10068000F000831626088400700880000230A50060
:10069000C830A40008000F302705013A8A110A1259
:1006A0000319602B0F302705023A8A110A12031D25
:1006B0000C2B031083161A1803148A110A12642BC8
:1006C0000310831619180314260884008001800D76
:1006D000840A80010230A500C830A4000800250863
:1006E000AF008A110A12AF1B0C2B8A110A12822149
:1006F0000530AE000800AE01AC012F08831696004D
:100700008A110A120319862B023097000800250867
:10071000013A8A110A12031D0C2BAD108A110A121C
:100720008221080025088A110A12031D0C2B2608B5
:10073000031D0C2B831603301705023A8A110A1287
:10074000031DAD2B83120F302705031DAD2B831620
:1007500018108A110A128221080083160330170527
:10076000033A8A110A12031D0C2B83120F3027053E
:10077000023C8A110A12031C0C2B83170F30270529
:100780008316983E840000108A110A128221080004
:100790008A110A120C2B2508013A8A110A12031D2C
:1007A0000C2BAD148A110A128221080025088A1127
:1007B0000A12031D0C2B2608031D0C2B8316033075
:1007C0001705023A8A110A12031DF12B83120F300A
:1007D0002705031DF12B831618148A110A12822192
:1007E0000800831603301705033A8A110A12031D05
:1007F0000C2B83120F302705023C8A110A12031CAE
:100800000C2B83170F3027058316983E84000014A5
:100810008A110A12822108008A110A120C2B8316EF
:1008200026088400831283172C0880008316013069
:10083000A500C830A40008002508013C8A110A124E
:10084000031C0C2B2508AC008A110A1203192B2C4F
:100850008316033097008A110A1282218316031728
:10086000C830AA000830A9008830A8000830AD00C0
:10087000D030AE004830AC00D830B2000830B10003
:100880008830B0000830B500D830B6004830B40029
:100890000E3099000E309A00080083161708033AAC
:1008A0008A110A12031D0C2B83122708003C8A119F
:1008B0000A12031C0C2B2708383E840083170008FB
:1008C000F000831626088400700880000130A5001F
:1008D000C830A40008008316170883120339033AAE
:1008E0008A110A12031D0C2B2708383E8400831737
:1008F000250880008A110A12822108008316031736
:1009000083172608840083120317B70137083502BE
:100910008A110A120319A02C8A110A12B40B932C03
:100920008A110A129F2C8A110A128D258000B70A9B
:10093000840A8A110A12B20F862CB30A862CAE01E1
:1009400037088316A5004030240640398838A400B3
:0A0950008A110A12080008000800CE
:06095A008A110A122308B5
:10096000213A0319D42C8A110A122308223A0319B6
:10097000712D8A110A122308233A0319712D8A1145
:100980000A122308A13A0319712D8A110A122308A9
:10099000A23A0319712D8A110A122308A33A0319E6
:1009A000712D8A110A120C2B2408013A8A110A129D
:1009B0000319712D2408023A8A110A120319712DA4
:1009C0002408033A8A110A120319712D2408063AE1
:1009D0008A110A120319012D2408093A8A110A12F0
:1009E0000319742D24080A3A8A110A120319712D69
:1009F00024080B3A8A110A120319712D8A110A125E
:100A00000C2B831203170630AE000830B500260801
:100A1000013A8A110A120319202D0310270D8A1199
:100A20000A128325B2000310270D013E8325B3006F
:100A30008A110A128D25B400B20A8A110A12402DB9
:100A40002608023A8A110A120319392D0310270DBC
:100A50008A110A128325B2000310270D013E832557
:100A6000B3008A110A128D25B400B20A8A110A1243
:100A7000402D2608033A8A110A1203190C2B08008C
:100A80002A088A110A12031D4A2D2908340229084E
:100A90000318B400B40A8A110A127E240800063032
:100AA000AE000830B500B730B2000530B3008A118F
:100AB0000A128D25B400AA088A110A12031D642D9A
:100AC00029022908031CB400B40A8A110A127E24E0
:100AD000080008008A110A122E08063A03197E241B
:100AE00008008A110A120C2B2130AE00831603175E
:100AF0000800F00005308A008130700703188A0A68
:100B00008200A5340534F00005308A008B30700770
:100B100003188A0A8200CE3405348312031733087F
:100B20008A00320882001234013400340134003467
:100B30000034003408340034003406340034003407
:100B400000340234013400340134093402342934CD
:100B50000034013401340434803432340934043430
:100B600000340034023403340034003400340934D7
:100B7000213400340134003401342234343400345C
:100B80000734053481340334083400340A3407341C
:100B9000053401340334083400340A343434063460
:100BA000A034FF3409340134A1340134093402344F
:100BB000A13400340634A134FF3409340334093439
:100BC00004341534803425347F34353400344534CE
:100BD000FF347534083495340834813402340934D0
:100BE0000534093406341534803425347F343534E3
:100BF00000344534FF347534083495340834913466
:100C00000234C034C0348312031733088A00320818
:100C10008200F0000310F00D8A110A121C26B600A3
:100C2000F00A8A110A121C26F00070088A003608A1
:100C3000330703188A0A820006308A0023307007BF
:100C400003188A0A820027340634333406343F34CA
:100C500006344534063467340634833406348F341E
:100C60000634993406343F340634A9340634BD348E
:100C70000634EB340634F7340634013407340634D2
:100C8000033409340434043408342234033449343A
:100C900000344F340034433400346134003472344F
:100CA0000034643400342D3400345534003453346B
:100CB00000344234003444340034433400346D345E
:100CC00000346F34003474340034723400341C3413
:100CD00003344D340034613400346E3400347534E0
:100CE0000034653400346C3400342034003456341D
:100CF0000034653400346C340034653400347A34A4
:100D00000034203400340C3403345634003431348D
:100D100000342E34003431340034303400340A349A
:100D200003344334003466340034673400343134DF
:100D30000034103403344E3400346F3400347434CF
:100D4000003468340034693400346E34003467345D
:100D50000034143403344D340034693400346334C3
:100D60000034723400346F34003463340034683437
:100D7000003469340034703400342E340334503479
:100D80000034693400346334003431340034363490
:100D900000344334003437340034363400343534CE
:100DA0000034203400345534003453340034423499
:100DB000003420340034493400344F340034433498
:100DC00000346134003472340034643400347334D9
:100DD0000034203400340C340334563400343134BD
:100DE00000342E34003430340034303400340A34CB
:100DF000033443340034663400346734003431340F
:100E00000034103403344E3400346F3400347434FE
:100E1000003468340034693400346E34003467348C
:020E200000349C
:101000001E30F200F20B02288316031381178A1593
:101010000A120623831603178A150A126400033086
:101020001705033A031D0E28831203138501860159
:1010300087018A150A128C218A150A12831323301C
:1010400084000830CC218A150A12031C1C28640075
:1010500083160313823081008030831203138100D2
:10106000831203138B178A150A12E1208B128A153B
:101070000A127121831203138B168A150A12831325
:10108000233084000830CC218A150A12031C4B2817
:101090008A150A12E1208312031381309F00BB21BD
:1010A0001F158A150A121F1951281E08A300B40023
:1010B000BB218312031389309F00BB211F158A15A2
:1010C0000A121F195F281E08A400BB2183120313F4
:1010D00099309F00BB211F158A150A121F196C2811
:1010E0001E08A500BB218312031391309F00BB2172
:1010F0001F158A150A121F1979281E08A600BB2180
:1011000083120313A1309F00BB211F158A150A12F9
:101110001F1986281E08A700BB218A150A128313EF
:101120008312031323308400083050228A150A12D8
:10113000031C8D288A150A12DB2883120313B601BB
:101140005030B700340837028A150A120318B02845
:10115000B500B509B50A8030B6008A150A12B12863
:10116000B5003508043C8A150A120318C32835084F
:101170001E3C8A150A120318C7284B303607A300F5
:101180008A150A12CB28A3018A150A12CB280A3025
:1011900036073507A300831203138B127D10FD1051
:1011A0002308AB00031DFD140330AB1BFD06AB137E
:1011B000831203138B168A150A12AA218A150A12A2
:1011C0003D28831203138B1283120313FD01FE01CA
:1011D0002308AB00031DFD140330AB1BFD06AB134E
:1011E0002408AC00031DFD150C30AC1BFD06AC1330
:1011F0002508AD00031DFD163030AD1BFD06AD13F7
:101200002608AE00031DFD17C030AE1BFD06AE1351
:101210002708AF00031DFE140330AF1BFE06AF13FB
:101220002808B000031D7E174430B01BFE06B01323
:10123000831203138B1608008A150A12F50303198B
:1012400047218A150A12F60303194E218A150A123C
:10125000F703031955218A150A12F80303195C21B3
:101260008A150A12F903031963218A150A12FA036F
:1012700003196A218A150A12F40B41298A150A12E8
:10128000712180308312031381000B110800FC30A0
:101290007B05FB008312031386000800F3307B05F7
:1012A000FB008312031386000800CF307B05FB0090
:1012B00083120313860008003F307B05FB00831276
:1012C000031386000800FC307C05FC008312031326
:1012D00087000800BB307C05FC00831203138700E5
:1012E00008007D08FB008312031386007E08FC00C3
:1012F000831203138700831203132B08F5002C08B5
:10130000F6002D08F7002E08F8002F08F900300825
:10131000FA007E30F400080083160313FF308500C6
:1013200000308600003087008316031302309F00D0
:10133000831203139F171F13831603130C138312B7
:101340000313A301A401A501A601A701A801A901F6
:10135000AA010800831203131430B800FF30B9004B
:10136000000000008A150A12B90BB0298A150A126A
:10137000B80BAE290800831203130230B800FF3007
:10138000B900000000008A150A12B90BC1298A159C
:081390000A12B80BBF29080086
:08139800030883120317C300D0
:1013A0000408BD00831603178A150A12A81B082A11
:1013B000290883120317C100C2008A150A120319F3
:1013C000F829831603172A0883120317BE00831710
:1013D0003E0884000008F1003D088400C31F831309
:1013E00071088000BD0ABE0A8A150A12C10BE729DE
:1013F000831628084039403A8838A8000830A900E8
:1014000083124208F10043088300710803140800A6
:101410008312031743088300031008000308831294
:101420000317C3000408BD00831603178A150A12A8
:10143000B01B4A2A310883120317C100C2008A1563
:101440000A1203193A2A8316031732088312031764
:10145000BE0083173E0884000008F1003D088400A8
:10146000C31F831371088000BD0ABE0A8A150A12C1
:10147000C10B292A831630084039403A8838B00019
:101480000830B10083124208F1004308830071085C
:101490000314080083120317430883000310080095
:1014A000F100030883120317C30071080F39C1004C
:1014B0000408BE004108831603178A150A12AC1BE4
:1014C000872AAD008A150A1203197B2A2E08831277
:1014D000BD008317C31F83133E0884000008F1007A
:1014E00083173D08840071088000BD0ABE0A8A1572
:1014F0000A12C10B692A83162C084039403A8838F1
:10150000AC00831203174308830003140800031080
:101510000800F100030883120317C30071080F3994
:10152000C1000408BE004108831603178A150A1279
:10153000B41BC02AB5008A150A120319B42A36084A
:101540008312BD008317C31F83133E088400000865
:10155000F10083173D08840071088000BD0ABE0AAF
:101560008A150A12C10BA22A831634084039403A60
:101570008838B4008312031743088300031408005B
:101580000310080083170339983E840000140800F4
:1015900083170339983E8400001008008312031754
:1015A000441C0800831610111115951463000000E7
:1015B0009510101211161011111108008312031743
:1015C000AD1C080083169510111610121111101180
:1015D00015158312BB018030BC008A150A12BB0BA3
:1015E000EF2ABC0BEF2A8316151108008316031788
:1015F00095118312BC01BB018A150A12BB0FFE2A8A
:10160000BC0FFE2A8A150A12062308008316031748
:101610009701013091009001083095008312AC01D0
:101620000130AD00B801B901BA01FF30AE0083123C
:1016300003138C1183168C150B178B170800831658
:0E164000031795119514970103138C110800E0
:044000000034003454
:02400E00FA3F77
:00000001FF
